S00C00006D61696E2E7372656373
S11300000C942A000C9445000C9445000C94450073
S11300100C9445000C9445000C9445000C94450048
S11300200C9445000C9445000C9445000C94470036
S11300300C9445000C9445000C9445000C94450028
S11300400C9445000C9445000C9445000C94450018
S11300500C94450011241FBECFE5D8E0DEBFCDBF10
S113006010E0A0E6B0E0EAE2F1E002C005900D92F3
S1130070A036B107D9F710E0A0E6B0E001C01D92A8
S1130080A536B107E1F70C947D000C9400001F9293
S11300900F920FB60F9211248F939F939091630048
S11300A09F5F909363009130A9F08091600098174E
S11300B009F4D89880916100981709F4D99880912F
S11300C06400981709F4DA9880916200981739F45B
S11300D0DB9805C0D89AD99ADA9ADB9AE6CF9F9131
S11300E08F910F900FBE0F901F90189581E083BFE2
S11300F089B7816089BF78940895CFE5D8E0DEBFE1
S1130100CDBF8FE08ABB17BA14BA11BA80E48093CA
S1130110600080E88093610080EF809364008FEF3B
S10D0120809362000E947600FFCF76
S9030000FC
